:040000008A01312917
:08000800F0000308F1000A08F2
:10001000F200831203138A110A128C1812280C188A
:1000200014282A298C102A290C1079308E00EC30E3
:100030008F00CC0A07305B06031D262896304C063D
:10004000031D26280714871407158715C8304C068A
:10005000031D2A29CC01DB0A08305B06031D392861
:10006000DB014A184A16CA18CA164A194A17CA1989
:10007000CA174818CD0AC818CE0A4819CF0AC81995
:10008000D00A78304D06031D7228CD0149184E283C
:1000900049143808C0003908C1007228D50A9630C2
:1000A000550603194B1403196C283908410203192A
:1000B0005C2803186C28492838084002031949288D
:1000C000031C4928D10A0230510603196C2838084C
:1000D000C0003908C1007228D1014A144810071025
:1000E000CD01D50178304E06031DA328CE01C918D5
:1000F0007F28C9143A08C2003B08C300A328D60AC7
:10010000963056060319CB1403199D283B08430269
:1001100003198D2803189D287A283A0842020319EA
:100120007A28031C7A28D20A0230520603199D2825
:100130003A08C2003B08C300A328D201CA14C81061
:100140008710CE01D60178304F06031DD428CF0189
:100150004919B02849153C08C4003D08C500D428F9
:10016000D70A9630570603194B150319CE283D08B8
:1001700045020319BE280318CE28AB283C084402C8
:100180000319AB28031CAB28D30A0230530603190A
:10019000CE283C08C4003D08C500D428D3014A1528
:1001A00048110711CF01D70178305006031D0529EA
:1001B000D001C919E128C9153E08C6003F08C7008B
:1001C0000529D80A963058060319CB150319FF28BC
:1001D0003F0847020319EF280318FF28DC283E08D0
:1001E00046020319DC28031CDC28D40A023054061A
:1001F0000319FF283E08C6003F08C7000529D4019F
:10020000CA15C8118711D001D8014B180B29481CF9
:100210000D29871F0D2987130E298717CB1814293D
:10022000C81C1629071F16290713172907174B196A
:100230001D29481D1F29871E1F298712202987165F
:10024000CB192629C81D2829071E28290712292964
:1002500007162A2972088A0071088300F00E700EB2
:1002600009008313203084008001840A841F34290C
:100270008316031380309F008312031381309F0085
:100280008312031385018601870179308E00EC30DB
:100290008F00353090008316031300308700FF3045
:1002A0008500FF3086008312031307148714071597
:1002B000871583160313573081008B170B1783168E
:1002C00003130C14831203131F156A216400CC213D
:1002D000640065291F190800831603131E08831282
:1002E0000313B50703110318B40A0319B30A1E0850
:1002F000B4070318B30AB60A0319B70A371DCA2987
:100300000A30B6000310B30CB40CB50CB603031DD1
:1003100082295908031D97299F15D90A3408B90065
:100320003508B8000A30DA00DA0B9429C5295908D3
:10033000013A031DA7299F111F16D90A3408BB00D3
:100340003508BA000A30DA00DA0BA429C5295908A1
:10035000023A031DB8299F111F129F16D90A3408AB
:10036000BD003508BC000A30DA00DA0BB529C52912
:100370009F111F129F12D9013408BF003508BE001B
:100380000A30DA00DA0BC229C817B301B401B5018B
:10039000B601B7011F150800C81F08000330390651
:1003A000031DD6290A3038020318DD294A1C4814D7
:1003B0004A1A07104A1A4A12E6294810CD01D501F7
:1003C00049104A1EE6294A124B104A1003303B06D8
:1003D000031DEE290A303A020318F529CA1CC81475
:1003E000CA1A8710CA1ACA12FE29C810CE01D6012D
:1003F000C910CA1EFE29CA12CB10CA1003303D060E
:10040000031D062A0A303C0203180D2A4A1D48150E
:100410004A1B07114A1B4A13162A4811CF01D7015C
:1004200049114A1F162A4A134B114A1103303F063D
:10043000031D1E2A0A303E020318252ACA1DC815AC
:10044000CA1B8711CA1BCA130800C811D001D801E2
:0E045000C911CA1F0800CA13CB11CA11080037
:02400E00B63DBD
:00000001FF
